:020000040000FA
:100000000128831203138501831606309F000030F8
:100010008500831286018316FF30860083128701D4
:100020008316FF30870083128501860187018501D1
:100030000430A000A00B1A28000005143A30A000DC
:10004000A00B202805100430A000A00B25280000DC
:1000500005143A30A000A00B2B2805100430A00096
:10006000A00B3028000005143A30A000A00B362861
:1000700005100430A000A00B3B28000005143A3006
:10008000A000A00B412805100430A000A00B4628BA
:10009000000005143A30A000A00B4C2805100430D5
:1000A000A000A00B5128000005143A30A000A00BBE
:1000B000572805103A30A000A00B5C280514043026
:1000C000A000A00B6128000005103A30A000A00B92
:1000D000672805140430A000A00B6C280000051050
:1000E0003A30A000A00B722805140430A000A00B29
:1000F0007728000005103A30A000A00B7D280514D9
:100100000430A000A00B8228000005103A30A000A7
:10011000A00B882805140430A000A00B8D28000037
:1001200005103A30A000A00B932805140430A0005D
:10013000A00B9828000005100430A000A00B9E28FA
:10014000000005143A30A000A00BA42805100430CC
:10015000A000A00BA928000005143A30A000A00BB5
:10016000AF2805100430A000A00BB428000005142F
:100170003A30A000A00BBA2805100430A000A00B54
:10018000BF28000005143A30A000A00BC5280510B8
:100190000430A000A00BCA28000005143A30A000CB
:1001A000A00BD02805100430A000A00BD52800001B
:1001B00005143A30A000A00BDB2805100830A00081
:1001C000A00BE028000005147530A000A00BE62865
:1001D00005100830A000A00BEB2805147530A00016
:1001E000A00BF02805100830A000A00BF52805147E
:1001F0007530A000A00BFA2805100830A000A00B55
:10020000FF2805147530A000A00B04290510083044
:10021000A000A00B092905147530A000A00B0E2921
:1002200005100830A000A00B132905147530A0009C
:10023000A00B182905100830A000A00B1D290514DB
:100240000D30A000A00B22290000051186018316A5
:100250000030860083122108870083160030870053
:100260008312210887008601000000008514860A99
:10027000860A860A860A860A860A860A860A860AFE
:10028000860A860A860A860A860A860A860A860AEE
:10029000860A860A860A860A860A860A860A860ADE
:1002A000860A860A860A860A860A860A860A860ACE
:1002B000860A860A860A860A860A860A860A860ABE
:1002C000860A860A860A860A860A860A860A860AAE
:1002D000860A860A860A860A860A860A860A860A9E
:1002E000860A860A860A860A860A860A860A860A8E
:1002F000860A860A860A860A860A860A860A860A7E
:10030000860A860A860A860A860A860A860A860A6D
:10031000860A860A860A860A860A860A860A860A5D
:10032000860A860A860A860A860A860A860A860A4D
:10033000860A860A860A860A860A860A860A860A3D
:10034000860A860A860A860A860A860A860A860A2D
:10035000860A860A860A860A860A860A860A860A1D
:10036000860A860A860A860A860A860A860A860A0D
:10037000860A860A860A860A860A860A860A860AFD
:10038000860A860A860A860A860A860A860A860AED
:10039000860A860A860A860A860A860A860A860ADD
:1003A000860A860A860A860A860A860A860A860ACD
:1003B000860A860A860A860A860A860A860A860ABD
:1003C000860A860A860A860A860A860A860A860AAD
:1003D000860A860A860A860A860A860A860A860A9D
:1003E000860A860A860A860A860A860A860A860A8D
:1003F000860A860A860A860A860A860A860A860A7D
:10040000860A860A860A860A860A860A860A860A6C
:10041000860A860A860A860A860A860A860A860A5C
:10042000860A860A860A860A860A860A860A860A4C
:10043000860A860A860A860A860A860A860A860A3C
:10044000860A860A860A860A860A860A860A860A2C
:10045000860A860A860A860A860A860A860A860A1C
:10046000860A860A860A860A860A860A8510860110
:100470008316FF308600831287018316FF308700C2
:10048000831205150530A000A00B442A8601482AD6
:10049000492AA10AFF3021020319172805101B2938
:02400E00BA3FB7
:00000001FF
